:100000003DC0000057C0000055C0000053C00000B4
:1000100051C000004FC000004DC000004BC00000A8
:1000200049C0000047C0000045C0000043C00000B8
:1000300041C000003FC000003DC0000033C10000CF
:1000400039C0000037C0000035C0000033C00000D8
:1000500031C000002FC000002DC000002BC00000E8
:1000600029C0000027C0000025C0000023C00000F8
:1000700021C000001FC000001DC0000011241FBED1
:10008000CFEFCDBFDFE3DEBF809140008093400023
:10009000811105C098ED21E094BF209341008CBBF5
:1000A00028E3A0E0B8E301C01D92AA30B207E1F74F
:1000B00028D179C1A5CF9FB7F89488E08093840AAE
:1000C00080918E0A81FFFCCF80918D0AE091A20A77
:1000D000F091A30A20910038309101384091023804
:1000E000509103389FBF80FF07C0E730F10520F42F
:1000F0002F5F3F4F4F4F5F4FBF0176956795CF0101
:10010000860F911DE62FE695E695762F72957F7006
:10011000E71BFF0B67FD3196E80FF91FA0E3B3E083
:1001200029D16E0F7F1F811D911D0895CF92DF92FF
:10013000EF92FF92CF93DF93BEDFEB0188EEC82EE4
:1001400083E0D82EE12CF12CB6DF6C1B7D0B683ED2
:100150007340A0F0C114D104E104F10439F4DF913B
:10016000CF91FF90EF90DF90CF90089581E0C81A73
:10017000D108E108F108C851DC4FE6CFC114D10421
:10018000E104F10409F7EBCFCF93DF93823108F05C
:1001900047C090E0EC01C052DC4728812F3F09F4B2
:1001A0003FC0AC0142535C47DA01EC91B0E2EB9FF7
:1001B000F0011124FC5F611136C0268330812323B6
:1001C000A1F49C0124543C47D9012C91309769F14A
:1001D000283058F57096E20FF11D3FB7F894208152
:1001E000611126C0277F20833FBF86559C47FC01B5
:1001F00090819923A9F08881903409F19038E1F039
:10020000903171F4DA019C919130A1F4853010F0B5
:10021000880F82959091010A809589238093010A25
:10022000DF91CF9108952583C9CFF0E0E0E0D5CFED
:100230002860D9CF880FEECF1092A006F1CF20E42E
:10024000823009F420E89091920A922349F36FB723
:10025000F8949091800A9E7F9093800A4091920A30
:1002600030E02095309550E02423352398ED94BF5D
:100270002093920A90918E0A90FFFCCF9091800A71
:1002800091609093800A813039F4809150048F7787
:10029000809350046FBFC4CF809151048F778093B7
:1002A0005104F8CF8F9381E080938D0A8FB78F939D
:1002B000EF93FF93E0E0F8E39F9368948FEF0DC016
:1002C000E89484819581805D9C4F84839583885ECA
:1002D000934080F0848395838FEF9081981B919356
:1002E00090819F4F919390819F4F919390819F4FC9
:1002F000919336F39F91FF91EF918F918FBF8F91E3
:10030000189588ED90E084BF90936100E0E0F6E0FE
:1003100083E582838DE0858380E2838381E080832F
:10032000109202028093030A9EEF9093260A909304
:10033000270A9BE09093000AE0E8FAE02DEF31E015
:1003400026A737A7118290E89283848781E1808372
:10035000789484E08093010480911204877F8093D5
:10036000120461E08FE010DFE1DE60E08FE00CDF7F
:10037000DDDEF7CF09D0A59F900DB49F900DA49F0F
:10038000800D911D11240895A29FB001B39FC0015B
:10039000A39F700D811D1124911DB29F700D811DB1
:0A03A0001124911D0895F894FFCF79
:1003AA0010108000000000101010404000000000F3
:1003BA0010000405060705040302010000010203F8
:1003CA000102030000000000010101010101020213
:1003DA0002020000000010204080201008040201E0
:0803EA000102040802040801ED
:00000001FF
